:1000000003308A00942B0000433BE1350D050000CE
:10001000E43777372A00F232671DA012CC3A0D057B
:1000200000002B30840083130008031924280230B9
:10003000F800F701F70B1A28F80B19289730F7008A
:10004000F70B2028800B17288A110A12212C8316FF
:100050008613831286130830F8002E280000F81744
:100060003F28F813B30C03188617031C8613781760
:100070003F287813F80B32283D28000086170230FD
:10008000F7008401840B4228F70B412823308400B9
:10009000840B48280000F81B3128781B39280800F9
:1000A000831603178C170C140000000083120C0831
:1000B0007F39031994280313AA0003170D080313AB
:1000C000AB0003170F080313AC002A08B300272066
:1000D0002B0803178D0003132C0803178F008316BA
:1000E0008C170C140000000083120C0D0E0D7F39CC
:1000F000031994280313AA0003170D080313AB0078
:1001000003170F080313AC002A08B30027202B089D
:1001100003178D0003132C0803178F008D0A031992
:100120008F0A031350280317031308008E30F700BB
:100130002B08F8002A08F900FA01F808031DAA287C
:100140007908F800F9010830F702F808031DAA2819
:10015000F701B2280310F81BB128F90DF80DF703C9
:10016000AA28F81308002A0803192329B2002E0828
:1001700003192329B2070318C4287F30B202031CD5
:10018000232903192329C8288130B20703182329FA
:100190003208F700F801F901FA012B08B600B6178A
:1001A0002C08B5002D08B4001830B200B301341C7F
:1001B000F1283108FA07031CE328F90A031DE32894
:1001C000F80A0319B3173008F907031CEA28F80ADC
:1001D0000319B3172F08AC00AC172C08F807031845
:1001E000B317B30DF80CF90CFA0CB60CB50CB40C33
:1001F0000310B20BD6280130F70703182329F81B88
:100200000829B60DFA0DF90DF80DF7030319232986
:10021000B61F1929FA0A031D1929F90A031D1929FC
:10022000F80A031D1929F80CF90CFA0CF70A03193E
:1002300023292B08B3002F08B306B31F2129F81771
:100240002729F8132729F701F801F901FA01080015
:1002500080308318B306B801B9012F08B7003308FE
:10026000B7062E080319182AB600F700320803193A
:10027000212AB6020319BD29031C7B293308BC00BF
:10028000BC173408BB003508BA00B9010310BC0C18
:10029000BB0CBA0CB90CB60B4529B71F5229381440
:1002A000352A3810361038163130840083134A2A24
:1002B0003812B71B6529361C7029BC0CBB0CBA0C54
:1002C000B90CF70A0319302A7029BC1B73290310D3
:1002D000B90DBA0DBB0DBC0DF7030319302A652902
:1002E0003817DD2938132F08B700B71F7929BC1735
:1002F000292ABC13292A3208B600F7002E08B602B4
:100300002F08BC00BC173008BB003108BA00B90187
:100310000310BC0CBB0CBA0CB90CB60B8729B71F69
:100320009429B814352AB8103610B8163530840020
:1003300083134A2AB812B71BA729361CB229BC0C52
:10034000BB0CBA0CB90CF70A0319302AB229BC1B32
:10035000B5290310B90DBA0DBB0DBC0DF703031978
:10036000302AA729B817DD29B8133308B700B71FFB
:10037000BB29BC17292ABC13292A3308BC00BC1787
:100380003408BB003508BA00B71FCA29BC1338159A
:10039000352A3811B90136103130840083134A2AC6
:1003A000B71BF3292F08B700361CDD29BC0CBB0C8A
:1003B000BA0CB90CF70A0319302AB91FEE29BA0A88
:1003C000031DEE29BB0A031DEE29BC0A031DEE29FD
:1003D000BC0CBB0CBA0CF70A0319302A381B722963
:1003E000B81BB429122A8030BC06BC1FFB29352A51
:1003F0003308B700082A2F08B700BC08031D082AD5
:10040000BB08031D082ABA08031D082AF701292A78
:10041000BC1B122A0310B90DBA0DBB0DBC0DF70B96
:10042000082A302AB71F162ABC17292ABC13292AE2
:100430003208F7003308BC003408BB003508BA00A6
:10044000292A2E08F7002F08BC003008BB0031080D
:10045000BA003C08F8003B08F9003A08FA00682A9C
:10046000F701F801F901FA01682AB901BA09BB09D3
:10047000BC09B909B90A031D432ABA0A031D432A54
:10048000BB0A0319BC0A38185129B818932938191E
:10049000C929F8290008BA07031C542ABB0A031DFE
:1004A000542ABC0A0319361484030008BB07031C32
:1004B0005C2ABC0A0319361484030008801F803AA2
:1004C000BC0703183614381A5829B81A9A29D029A3
:1004D00008000408F800831606178312061B6E2A0C
:1004E0000830F700AA01F717852AF713852A0310A9
:1004F000061B0314AA0C7717852A7713F70B772AA4
:10050000780884002A08F8009A2A02308400003013
:10051000F71B5530F800F80B8B2A840B872A213003
:10052000F71B0930F800F80B932AF71B752A771B85
:100530007D2A772A8A110A12762C831603178C17C4
:100540000C14000000000318CC2A83120C087F3919
:100550000313AB0003170D080313AC0003170F08B8
:100560000313AD002B08B30027202C0803178D00C0
:1005700003132D0803178F0083168C170C1400002B
:10058000000083120313AA0BC62AC92A8316031775
:10059000CC2AEB2A8316031783120C0D0E0D7F391C
:1005A0000313AB0003170D080313AC0003170F0868
:1005B0000313AD002B08B30027202C0803178D0070
:1005C00003132D0803178F008D0A03198F0A0310D8
:1005D0000313AA0B9D2A8A110A12F12CB2010408F6
:1005E000B1003210831B32142B0EF038AD00AD0772
:1005F000E23EAE00323EB0002B080F39AE07AE0728
:10060000B007E93EAF00AF07AF072A0E0F39AF07BB
:10061000B007AF0DB00DB009B00D2A080F39B00703
:10062000AD0D0730AC000A30B007AF03031C142B2C
:10063000AF07AE03031C182BAE07AD03031C1C2B26
:10064000AD07AC03031C202B2C3084008313073030
:1006500031053113840730300402031931170008C3
:10066000F700031D3B2B311B3B2B311A4D2BB119CE
:100670003B2B20303E2BB11531123030F707AB0148
:100680000408AA002B10831B2B147708B300272023
:100690002A08840083132B188317840A311F2B2BFD
:1006A0008A110A12F82C2B08B2002F08B206B21FCA
:1006B0005E2B03110310AB1B0314912B2B08B2000C
:1006C0002E08B3002A08B30203196C2BB21F912B1A
:1006D0000308013A8300912B2F08B3002B08B302C3
:1006E0000319782BB21F912B0308013A8300912B39
:1006F0003008B3002C08B3020319842BB21F912BCE
:100700000308013A8300912B3108B3002D08B3028E
:100710000319902BB21F912B0308013A8300912BF0
:1007200003108A110A12142D840183131F308305CC
:10073000713083168F000F08861383128617831675
:1007400003170908C039890003131F129F120030D4
:10075000031788008312870188018901FF30031382
:10076000A000831603170908C039890003131F125C
:100770009F12013003178800831203131F139F1366
:1007800083169F1783121F149412A0122008831639
:100790008700831220162008831687008312A01179
:1007A00020088316870001308312940000308316DE
:1007B00094000108C7390838810083129001003085
:1007C000F8000438920063308316920083122011DF
:1007D00020088316870083120711831609130C3033
:1007E0008312970083169B019C0101309D008312A8
:1007F000A010200883168700831287100C309D00FC
:1008000001308000323095001708CF3997006430EE
:100810009B001D08CF399D000317870188018901BE
:100820007130831603138F000F080030F800831215
:100830001F08C33978049F000230AA00FA30AB00C9
:100840001128AA0B1E2C043003178D0000308F00D6
:10085000031350200130A2009030A1002208AB0009
:100860002108AA009620AE30AD004730AC00013020
:10087000AB008030AA007A08B1007908B00078088F
:10088000AF007708AE00B3207708AA007808AB0065
:100890007908AC007A08AD0083107A08B1007908B5
:1008A000B0007808AF007708AE00B5018030B40022
:1008B000E130B3008730B20028217A08A600790819
:1008C000A5007808A4007708A3009F149F18662C41
:1008D00083161E088312A7001E08A800061BFE2C04
:1008E00064309B001D08CF399D00692A7808A90053
:1008F0002908753C031D922C2208023C031C892CFC
:10090000031D862C2108573C031C892CA10A0319BE
:10091000A20A7530B30027207030B30027202A3098
:10092000B30027202908643C031DA82CA208031D3E
:100930009D2C2108FA3C0318A12C21080319A203BD
:10094000A103083003178D0000308F0003135020DF
:100950002908603C0318FE2C29087A3C031CFE2C55
:100960002208AB002108AA009620AE30AD00473027
:10097000AC000130AB008030AA007A08B1007908E1
:10098000B0007808AF007708AE00B3207708AA005F
:100990007808AB007908AC007A08AD0083107A08BB
:1009A000B1007908B0007808AF007708AE00B50153
:1009B0008030B400E130B3008730B20028217A08DB
:1009C000A6007908A5007808A4007708A3000B30DA
:1009D00003178D0000308F00031005300313AA00A9
:1009E0009D2A103084002208AB002108AA00EE2ABC
:1009F0000D30B30027200A30B30027202808AB00B1
:100A00002708AA0096202608AD002508AC00240877
:100A1000AB002308AA007A08B1007908B000780872
:100A2000AF007708AE00532B0318182D031D1E2DA1
:100A300064309B001D08CF399D00242D3F309B0062
:100A40001D08CF3930389D008530F700F70B262D73
:040A5000652C6300AE
:04400E00F52CFF3F4F
:00000001FF
